:020000040000FA
:10000000C828FF3FFF3FFF3F8B0109009401051106
:10001000940B0B28080005150000072894011028F0
:100020000511940B142808000515162800000F2848
:10003000940122200511940B1E280800051522208A
:10004000000019280800AE0051302E020800AE0052
:1000500003102E0C0800AE0011302E020800AE0076
:100060000310AE0C03102E0C0800AE0002302E0759
:100070000800182006200E2008000620A4200620D4
:10008000A42018200800971644309600861B08000C
:10009000960B4628971208000617FE30AA00031494
:1000A000AA0D2A1F5D282A0886054320971E4F287F
:1000B00086012A0986049E045E2886010613A42070
:1000C0000800073089009B200808A200890A9B20AD
:1000D0000808A300890A9B200808A900A21222137D
:1000E000A2132310A31008000730890022088800FB
:1000F0008220890A230888008220890A290888002A
:10010000822008008316081208158B1355308900C9
:10011000AA30890088140811081E8C288312080848
:100120008316081483120802031906200800110818
:1001300089008220080083160814831208002930E1
:100140009600960BA1280800A4309600960BA628CE
:1001500008001430AB00A420AB0BAB280800A9208A
:100160000515A9200511A42005159F209F20051124
:10017000A420080026309600960BBC280000000042
:10018000080011306500803066008330620008008E
:10019000C1203E3086040613851185100610051116
:1001A0008B01831688018301223089009E0197010B
:1001B000A601A80101309E059D01861FE2280518B1
:1001C0007F2AC8286120960101309000861BC8282C
:1001D00005187F2A960BE628900BE6284C20910103
:1001E0001A3084008403A617CE2A6120051A11292B
:1001F0001E1DFD28231D11290E299E1C0229A31D49
:1002000011290E299E1D0729231E11290E291E1EA4
:100210000C29A31E11290E29231F112917150617B2
:10022000A4011030AC00AB01C1208511851006146B
:1002300005111A29861F14299F20861F1429A61329
:1002400090010B3010020319C828100803192B293C
:100250009F20861F3629900A8101861F3429CE30BF
:100260000102031C2D29C8289F208101861B2129FA
:10027000CE300102031C3629171A372B9719482A4A
:10028000261B3B2A1E1B6A2997186F29971BDE2AFB
:100290001C300402031C840A10088000910A0330F9
:1002A00011020319592A171F142905301102031DC1
:1002B00014291713023035200002031D142984036A
:1002C0000C302F200002031D14291E17A612062031
:1002D000A42014291E131008A50097141429250E14
:1002E00090079710910121301002031D792997156D
:1002F000142922301002031D81299E17103091000D
:10030000772923301002031D8829261513307F29F1
:1003100024301002031D8F29A61516307F292530A1
:100320001002031D962926161A307F29313010023B
:10033000031DA129A3112213A61EA315A61A221775
:10034000F02932301002031DA829A3112213F0292D
:1003500033301002031DB3292311A212A61E231548
:10036000A61AA216F02934301002031DBA2923114F
:10037000A212F02935301002031DC5292312A21341
:10038000A61E2316A61AA217F02936301002031D46
:10039000CC292312A213F02937301002031DD729CC
:1003A000A3122310A61EA316A61A2314F029383070
:1003B0001002031DDE29A3122310F0293930100288
:1003C000031DE9292313A310A61E2317A61AA3149D
:1003D000F0294A301002031DF2292313A310F0293B
:1003E0007420142945301002031DF929A6161E1782
:1003F000142943301002031DFF29261714295130F8
:100400001002031D052A2214F02952301002031D88
:100410000B2A2210F02953301002031D112AA214B6
:10042000F02954301002031D172AA210F02955306C
:100430001002031D1D2A2215F02956301002031D3B
:10044000232A2211F02957301002031D292AA21550
:10045000F02958301002031D2F2AA211F02959301B
:100460001002031D352A2216F0296A301002031DDE
:10047000F1292212F02926130A301002031D422A04
:10048000FF30432A100888001E308900822014297A
:1004900003309E1B133026191630A6191930261A60
:1004A0001D30110203181429100888009720910AA2
:1004B00014291A3084000230840716302B200002E1
:1004C000031D732A8403023027200002031D732AB0
:1004D0008403533023200002031D732A1A30840042
:1004E0008403171714291A30023E8400142981014D
:1004F000051C942ACE300102031C782A9C2AA21CD7
:100500000611221C8610221D8611A21D0612221E13
:100510008612061499019D0161201E3089009B20DE
:10052000C120051C942A902A8101990A0518772A6E
:10053000CE300102031C962A033019020318A42AA4
:100540009D08031DAE2AC8289D0A08081D02031D28
:10055000AE2A0615861486150616861632309000C9
:10056000910199010518902A861FBB2A910BB22A86
:10057000900BB22AC828960103309200861BB62A37
:100580000518902A960BBE2A920BBE2A1716053024
:100590009200A420920BC92A4C200617051AD52ACE
:1005A00097179101A61F1429F5289701A601A80104
:1005B000061797131A3084008403D12ADF2A910A80
:1005C0001719002B1E1DE62A1429F42A9E1CE92A5D
:1005D00014299E1DEC2A14291E1EF02A231C1429FE
:1005E0009E1EF42AA31C142901301102031D142994
:1005F00008301002031D142917150617A401142929
:1006000000301E1910309E1913301E1A16309E1A13
:100610001A309400A40A01302402031D162B14087A
:1006200089009B2008081002031D352B023024028C
:10063000031D212B140A89009B2008081002031DAA
:10064000352B03302402031D1429940A140A89004F
:100650009B2008081002031D352B17110613A42038
:10066000A4203D20A42097171429171114298515BB
:100670003920A610C130860501301002031D472B1A
:1006800086149D23971A862B9E019E14722B02308E
:100690001002031D522B06159D23971A862B9E01CF
:1006A0001E15722B03301002031D5D2B86159D2332
:1006B000971A862B9E019E15722B04301002031D83
:1006C000682B06169D23971A862B9E011E16722BE9
:1006D00005301002031D832B86169D23971A862B47
:1006E0009E019E16A4201429171217107823722B2E
:1006F0001E1906159E1886149E1986151E1A0616B2
:100700009E1A861608003E30860414291718982B66
:10071000A618C828C1308605A6141E194B2B9E1892
:10072000402B9E19562B1E1A612B9E1A6C2BC82823
:10073000782306200E201820C82897128515061346
:100740001030A700A420A70BA22B1430A7001A304A
:100750009100851405110610BA2006140515000035
:100760000000BA20910BAA2B05118510A70BB92BFD
:10077000C72B043091009001861FCB2B85150613E3
:10078000900BBC2B910BBC2B85150613A72B971632
:100790000617851108009601013090000617851193
:1007A000861BBE2B960BCE2B900BCE2B8511910169
:1007B000061708001430A100A420A10BDC2B0800B0
:1007C000FF3FFF3FFF3FFF3FFF3FFF3FFF3FFF3F39
:1007D000FF3FFF3FFF3FFF3FFF3FFF3FFF3FFF3F29
:1007E000FF3FFF3FFF3FFF3FFF3FFF3FFF3FFF3F19
:1007F000FF3FFF3FFF3FFF3FFF3FFF3FFF3FFF3F09
:08400000FF3FFF3FFF3FFF3FC0
:02400E00F03F81
:00000001FF
